BL51 BANKED LINKER/LOCATER V6.00                                                        10/29/2010  14:06:14  PAGE 1


BL51 BANKED LINKER/LOCATER V6.00, INVOKED BY:
C:\KEIL\C51\BIN\BL51.EXE STARTUP.obj, chengxu.obj TO chengxu RAMSIZE (256)


MEMORY MODEL: SMALL


INPUT MODULES INCLUDED:
  STARTUP.obj (?C_STARTUP)
  chengxu.obj (CHENGXU)


LINK MAP OF MODULE:  chengxu (?C_STARTUP)


            TYPE    BASE      LENGTH    RELOCATION   SEGMENT NAME
            -----------------------------------------------------

            * * * * * * *   D A T A   M E M O R Y   * * * * * * *
            REG     0000H     0008H     ABSOLUTE     "REG BANK 0"
            IDATA   0008H     0001H     UNIT         ?STACK

            * * * * * * *   C O D E   M E M O R Y   * * * * * * *
            CODE    0000H     0003H     ABSOLUTE     
            CODE    0003H     000FH     UNIT         ?PR?MAIN?CHENGXU
            CODE    0012H     000DH     UNIT         ?PR?DELAY?CHENGXU
            CODE    001FH     000CH     UNIT         ?C_C51STARTUP



OVERLAY MAP OF MODULE:   chengxu (?C_STARTUP)


SEGMENT
  +--> CALLED SEGMENT
---------------------
?C_C51STARTUP
  +--> ?PR?MAIN?CHENGXU

?PR?MAIN?CHENGXU
  +--> ?PR?DELAY?CHENGXU



SYMBOL TABLE OF MODULE:  chengxu (?C_STARTUP)

  VALUE           TYPE          NAME
  ----------------------------------

  -------         MODULE        ?C_STARTUP
  C:001FH         SEGMENT       ?C_C51STARTUP
  I:0008H         SEGMENT       ?STACK
  C:0000H         PUBLIC        ?C_STARTUP
  D:00E0H         SYMBOL        ACC
  D:00F0H         SYMBOL        B
  D:0083H         SYMBOL        DPH
  D:0082H         SYMBOL        DPL
  N:0000H         SYMBOL        IBPSTACK
BL51 BANKED LINKER/LOCATER V6.00                                                      10/29/2010  14:06:14  PAGE 2


  N:0100H         SYMBOL        IBPSTACKTOP
  N:0080H         SYMBOL        IDATALEN
  C:0022H         SYMBOL        IDATALOOP
  N:0000H         SYMBOL        PBPSTACK
  N:0100H         SYMBOL        PBPSTACKTOP
  N:0000H         SYMBOL        PDATALEN
  N:0000H         SYMBOL        PDATASTART
  N:0000H         SYMBOL        PPAGE
  N:0000H         SYMBOL        PPAGEENABLE
  D:00A0H         SYMBOL        PPAGE_SFR
  D:0081H         SYMBOL        SP
  C:001FH         SYMBOL        STARTUP1
  N:0000H         SYMBOL        XBPSTACK
  N:0000H         SYMBOL        XBPSTACKTOP
  N:0000H         SYMBOL        XDATALEN
  N:0000H         SYMBOL        XDATASTART
  C:0000H         LINE#         126
  C:001FH         LINE#         133
  C:0021H         LINE#         134
  C:0022H         LINE#         135
  C:0023H         LINE#         136
  C:0025H         LINE#         185
  C:0028H         LINE#         196
  -------         ENDMOD        ?C_STARTUP

  -------         MODULE        CHENGXU
  C:0000H         SYMBOL        _ICE_DUMMY_
  D:0090H         PUBLIC        P1
  D:00A0H         PUBLIC        P2
  D:00B0H         PUBLIC        P3
  D:00A8H         PUBLIC        IE
  C:0012H         PUBLIC        delay
  D:00B8H         PUBLIC        IP
  C:0003H         PUBLIC        main
  D:0098H         PUBLIC        SCON
  D:0088H         PUBLIC        TCON
  B:00A0H.0       PUBLIC        DOUT
  B:0090H.0       PUBLIC        LED
  D:00C8H         PUBLIC        T2CON
  D:00D0H         PUBLIC        PSW
  -------         PROC          DELAY
  -------         DO            
  D:0007H         SYMBOL        m
  D:0006H         SYMBOL        n
  D:0005H         SYMBOL        s
  -------         ENDDO         
  C:0012H         LINE#         28
  C:0012H         LINE#         29
  C:0012H         LINE#         31
  C:0014H         LINE#         32
  C:0016H         LINE#         33
  C:001EH         LINE#         34
  -------         ENDPROC       DELAY
  -------         PROC          MAIN
  C:0003H         LINE#         38
  C:0003H         LINE#         39
  C:0003H         LINE#         40
BL51 BANKED LINKER/LOCATER V6.00                                                      10/29/2010  14:06:14  PAGE 3


  C:0003H         LINE#         41
  C:0003H         LINE#         42
  C:0005H         LINE#         43
  C:0008H         LINE#         44
  C:0008H         LINE#         45
  C:000BH         LINE#         46
  C:000EH         LINE#         47
  C:000EH         LINE#         48
  C:0010H         LINE#         49
  C:0010H         LINE#         50
  C:0010H         LINE#         51
  -------         ENDPROC       MAIN
  -------         ENDMOD        CHENGXU

Program Size: data=9.0 xdata=0 code=43
LINK/LOCATE RUN COMPLETE.  0 WARNING(S),  0 ERROR(S)
